:020000040000FA
:020000000428D2
:08000800FF30A100FF30A2004F
:1000100021103C2023103B2019301A2024143420B6
:100020002514332019301A202410342025103320B1
:100030000C281928A6002608A7006430A800013063
:100040002128A900FF30AA002808AC002708AB002F
:1000500077302A0703182928AB0B2828AC0B262851
:10006000A90B24280800352838282508870008000F
:100070002408850008003D28402823086700080060
:06008000210865000800E4
:044200000C000F009F
:02400E00C211DD
:00000001FF
